:1000000092C0A6C6ABC0AAC0A9C0A8C0A7C0A6C0BF
:10001000A5C02FC8A3C0A2C0A1C0A0C09FC09EC041
:100020009DC09CC09BC000000001010203030405A9
:100030000506070708090A0A0B0C0D0D0E0F101113
:10004000121213141516171818191A1B1C1D1E1F2F
:1000500020212122232425262728292A2B2C2D2E36
:100060002F303132333435363738393A3B3C3D3E28
:100070003F4041424345464748494A4B4C4D4E4F0D
:100080005051535455565758595A5B5D5E5F6061E5
:10009000626364666768696A6B6C6E6F70717273B5
:1000A00075767778797A7C7D7E7F8081838485867A
:1000B00087898A8B8C8D8F90919294959697989A38
:1000C0009B9C9D9FA0A1A2A4A5A6A7A9AAABACAEEC
:1000D000AFB0B1B3B4B5B6B8B9BABBBDBEBFC1C29B
:1000E000C3C4C6C7C8CACBCCCDCFD0D1D3D4D5D743
:1000F000D8D9DADCDDDEE0E1E2E4E5E6E8E9EAECE5
:10010000EDEEF0F1F2F4F5F6F8F9FAFCFDFEFFFF82
:10011000FFFFFFFFFFFFFFFFFFFFFFFFFFFFFFFFEF
:10012000FFFFFFFFFFFF11241FBECFE5D4E0DEBFBE
:10013000CDBF11E0A0E6B0E0E8ECF6E102C005902A
:100140000D92A837B107D9F724E0A8E7B1E001C0C4
:100150001D92AB34B207E1F735D9B4CA51CF9091B3
:100160004602911105C028EA31E640E050E005C0A2
:100170009CE028E431E740E050E06058A62FBB2720
:10018000A7FDB095A81BB10987FDB3959923F9F098
:100190001A161B0654F4892F992787FD9095A817E6
:1001A000B9079CF0A81BB90B12C0109781F0892FDA
:1001B000992787FD909566277727681B790B6A1723
:1001C0007B071CF0A80FB91F02C0A0E0B0E002DA64
:1001D00020E03DE740E050E0DBD9C90182382FEF55
:1001E000920724F08038910524F4089581E89FEF68
:1001F00008958FE790E00895019728E3289FD001A4
:10020000299FB00D1124A95BBD4F88E3E6E0F2E021
:1002100001900D928A95E1F75AC72F923F924F9223
:100220005F926F927F928F929F92AF92BF92CF9286
:10023000DF92EF92FF920F931F93CF93DF9300D043
:100240001F92CDB7DEB710910402812F8071809389
:10025000AF00812F88708093B300812F80788093C6
:10026000B700812F81708093BB00812F80728093B3
:10027000BF00812F80748093C30000910102005859
:100280000093C7000093CB008091000280588983BF
:100290008093CF008093D30080910502982F9170B6
:1002A0009093D700982F92709093DB00982F9870BE
:1002B0009093DF0084708093E300F090FF016091E1
:1002C000FE0180917D014BDF5C016F2D80917C01EF
:1002D00046DF9B838A839C0197FF03C0319521955C
:1002E00031091501B7FE04C0222433242A183B0823
:1002F0006501EE24D7FCE094FE2C30E0D50164D9F2
:10030000412C42E0542E612C712CA301920140D962
:10031000C20ED31EE41EF51EEA81FB814F01AA2402
:1003200097FCA094BA2C222D30E0DF014DD9A30117
:1003300092012ED9820E931EA41EB51EF2E8CF168E
:10034000FFEFDF06EF06FF0664F080E8C816D10471
:10035000E104F10464F02FE7C22ED12CE12CF12C42
:1003600006C031E8C32EDD24DA94ED2CFD2C92E892
:1003700089169FEF9906A906B90664F0E0E88E1683
:100380009104A104B10464F08FE7882E912CA12C74
:10039000B12C06C091E8892E99249A94A92CB92CE5
:1003A000C092E7008092EB00812F84708093EF0071
:1003B00012701093F3008092F7008092FB00C092BD
:1003C000FF00C092030180910202805880930701D0
:1003D00080910302805880930B01F981F0930F0103
:1003E000009313010F900F900F90DF91CF911F9109
:1003F0000F91FF90EF90DF90CF90BF90AF909F90C4
:100400008F907F906F905F904F903F902F900895C6
:100410008FEF99EF0197F1F700C00000E091FC0128
:10042000F091FD010484F585E02D80E00995E091CF
:10043000FC01F091FD010684F785E02D09958823E4
:1004400039F3E091FC01F091FD010088F189E02D84
:100450008EEF91E00995E1DE91E080E02091AF0020
:10046000211101C090E0292F382F8091B300811114
:1004700022608091EF00811124608091F30081114E
:1004800028608091B700811120618091BF008111A7
:1004900020628091C300811120648091D700811176
:1004A00020688091DB00811131608091DF00811133
:1004B00032608091E300811134608091BB00811132
:1004C000386060917A0170917B01622773274CE05C
:1004D00050E081E090E0FC01E623F723EF2B51F0A0
:1004E000FC01E223F323EF2B29F030937B012093CF
:1004F0007A010895880F991F4150510941155105FE
:1005000051F730937B0120937A0182CF9C012150D7
:1005100031092430310508F46FCE089528E3E0E670
:10052000F0E0A6E0B2E001900D922A95E1F7019784
:1005300084309105D8F448E3489F9001499F300DDD
:100540001124F901E95BFD4FD901A25CBD4F199659
:100550008C918F3F41F088E3A6E0B2E001900D92CC
:100560008A95E1F703C08FEF9FEF089580E090E058
:10057000089581E090914602911180E080934602B7
:10058000A6C580934502A3C5EF92FF920F931F93D8
:10059000CF93DF9300D01F92CDB7DEB78B018032AF
:1005A000910519F07B0120E81DC0FB01808191813C
:1005B0008F3FFFEF9F0709F453C00196FB014DC029
:1005C000893091059CF48230910599F18430910530
:1005D000A1F1019759F129834A835B8319DF5B817C
:1005E0004A8129818830910559F72BC080329105C5
:1005F00061F18115F8E09F0799F1409761F7203884
:1006000041F0822F90E0F701918380837A0120E806
:10061000E2CFF801808191818F3FFFEF9F0701F1C9
:100620000196F801918380837A01D5CF220F220FA2
:10063000D2CF220F220F2F5FCECF220F220F2E5F9D
:10064000CACF220F220F2D5FC6CFE016F10641F070
:10065000203849F0822F90E0F7019183808303C016
:100660008FEF9FEF02C080E090E00F900F900F900F
:10067000DF91CF911F910F91FF90EF90089581E04E
:1006800090E0D5D4C5DE811522E09207A9F044F4AC
:100690008038910579F081159140B9F482E00FC05E
:1006A000811524E0920751F08115984071F4109261
:1006B000450207C081E003C083E001C084E080936D
:1006C000450205D580E090E008958FEF9FEF0895F3
:1006D00081E090E0ACD49CDE811521E09207E1F04E
:1006E00054F48032910529F18038910591F04097BA
:1006F00009F53FDF17C0811524E0920781F08115CD
:1007000028E0920791F081159240A1F483E090E0F7
:1007100008C081E090E005C082E090E002C084E083
:1007200090E06ADD80E090E0089580E090E0F6DE01
:10073000F9CFA5CF8FEF9FEF0895FF920F931F93EF
:10074000CF93DF9300D000D0CDB7DEB78FEF9FEF10
:100750009C838B839A838983FFB6F89465D485E064
:1007600090E065D4E091FC01F091FD010484F585F1
:10077000E02D80E00995E091FC01F091FD010088F9
:10078000F189E02D8EEF91E0099547DD8091BB0066
:10079000882339F08FEF99EF0197F1F700C000003F
:1007A000E1CF01E010E034DE80329105D9F194F41C
:1007B00084309105B9F13CF49C012150310922307B
:1007C000310588F72FC08830910561F1803191059E
:1007D00051F728C0811521E09207C9F04CF480340C
:1007E0009105E1F080389105F1F681E090E014C0C8
:1007F000811524E0920771F0811528E0920709F431
:1008000047C08115924079F683E090E005C082E010
:1008100090E002C084E090E081DE01C059DF0196E3
:10082000B9F523C0AE014F5F5F4FBE016D5F7F4FD3
:10083000ABDE0196D1F08B819C810196B1F089816C
:100840009A81019691F0012B19F080E090E066DE2C
:1008500049815A816B817C8186E092E051D381E0AD
:1008600090E0E5D300E010E09ECF83E090E0DFD39E
:1008700081E090E0F9D38FEF9DE222E28150904039
:100880002040E1F700C0000080E090E0EDD303C01D
:1008900083E090E0CCD34AD4FFBE0F900F900F902E
:1008A0000F90DF91CF911F910F91FF900895FC0160
:1008B0008585882391F001D4882399F0809178016F
:1008C0009091790101969093790180937801069730
:1008D00044F033DF81E090E00895109279011092A6
:1008E000780180E090E008959B01285F3F4F90E8F9
:1008F000492F4823FB014193BF019695E217F30767
:10090000B9F708951F93CF93DF93FC01EB0181E0CA
:1009100021819381291301C080E0888381E02581B2
:100920009781291301C080E0898381E02185938527
:10093000291301C080E08A8381E0258597852913EA
:1009400001C080E08B8381E021A593A5291301C01C
:1009500080E08C8381E025A597A5291301C080E064
:100960008D8381E021A993A9291301C080E08E83A2
:1009700081E025A997A9291301C080E08F831886FB
:10098000198681E021899389291301C080E08A8733
:1009900081E025899789291301C080E08B8781E058
:1009A000218D938D291301C080E08C8781E0258DF6
:1009B000978D291301C080E08D8781E021A193A14B
:1009C000291301C080E08E8781E025A197A129131A
:1009D00001C080E08F8721AD95ADDF01A05CBF4FE6
:1009E00011968C91119713963C91831301C0892F16
:1009F000DF01AC5BBF4F11961C91119713969C9130
:100A0000191301C0182FDF01A85BBF4F11969C91ED
:100A1000119713968C91981301C0922FE45BFF4FAE
:100A200081812381821301C0892FBE01605F7F4FC6
:100A30005BDFBE01685E7F4F812F8095DF91CF9194
:100A40001F9152CF009741F028E0E6E8F1E0DC0189
:100A500001900D922A95E1F788E0E6E8F1E0AEE733
:100A6000B1E001900D928A95E1F708958091980088
:100A700090919900892B31F0109299001092980072
:100A800081E0089548E050E06EE771E086E891E08B
:100A9000DFD50895CF93DF93CDB7DEB728970FB694
:100AA000F894DEBF0FBECDBFFE01319688E0DF01B6
:100AB0001D928A95E9F7698180E090E020E830E0B6
:100AC000DC01A95ABC4F4C91442341F0A901082EE6
:100AD00002C0559547950A94E2F701C040E0462BC5
:100AE00001968830910511F0642FEACF49836A811D
:100AF00080E090E020E830E0DC01A15ABC4F4C914E
:100B0000442341F0A901082E02C0559547950A9447
:100B1000E2F701C040E0462B01968830910511F0C4
:100B2000642FEACF40954A836B8180E090E020E813
:100B300030E0DC01A959BC4F4C91442341F0A9019C
:100B4000082E02C0559547950A94E2F701C040E08F
:100B5000462B01968830910511F0642FEACF4B8324
:100B60006C8180E090E020E830E0DC01A159BC4FCE
:100B70004C91411108C0A901082E02C05595479516
:100B80000A94E2F701C040E0462B019688309105B7
:100B900011F0642FEACF4C836D8180E090E020E873
:100BA00030E0DC01A958BC4F4C91442341F0A9012D
:100BB000082E02C0559547950A94E2F701C040E01F
:100BC000462B01968830910511F0642FEACF4095AD
:100BD0004D836E8180E090E020E830E0DC01A15898
:100BE000BC4F4C91442341F0A901082E02C05595F9
:100BF00047950A94E2F701C040E0462B0196883001
:100C0000910511F0642FEACF40954E833F8180E03B
:100C100090E041E0DC01A65BBC4F2C91222339F02F
:100C2000242F082E01C0220F0A94EAF701C020E009
:100C3000322B01968530910569F780915003882306
:100C400011F080E201C080E0382B809151038823AD
:100C500011F080E401C080E0382B8091520388239A
:100C600011F080E801C080E0382B3F83288580E0C8
:100C700090E051E0DC01AD5ABC4F4C91442339F077
:100C8000452F082E01C0440F0A94EAF701C040E046
:100C9000242B01968430910569F72887A6E8B1E0F6
:100CA000CE01079641914D93E817F907D9F7309394
:100CB0008C0120938D0128960FB6F894DEBF0FBEED
:100CC000CDBFDF91CF910895CF93DF93CDB7DEB73E
:100CD00029970FB6F894DEBF0FBECDBF198661E02D
:100CE00070E0CE0109969BD28831A9F487EC90E0A0
:100CF0000197F1F700C0000080E4898383E08A83D4
:100D00001B8263E070E0CE01019689D2803419F431
:100D1000C1DE80E001C081E029960FB6F894DEBF05
:100D20000FBECDBFDF91CF91089581E0CDDF91E07F
:100D3000811190E0892F08958FB7F894B99AC198DE
:100D4000A398AB988FBF81E0BFCF8AE990E0089568
:100D50001F921FB6EF93FF934F930F931F937F93B1
:100D6000EEE8F1E009E00EC016E01A95D1F040B3CC
:100D70004470D9F7000000000000000000000000EF
:100D8000000000002ED0000040B3000044704193EA
:100D90000A9539F015E11A9521F040B34470D9F362
:100DA000E3CFEEE8F1E040814423B9F447814423E6
:100DB000B1F059D005C0909A00000000909800C092
:100DC00041E0E5EFF1E040837F911F910F914F915A
:100DD000FF91EF911FBE1F90189532D0F1CF1DD01B
:100DE000EFCF12E01A95F1F708950F931F93442760
:100DF00000E81191112309F0402B0695D1F71F91BE
:100E00000F9108950F931F9300E8142F102311934F
:100E10000695D9F71F910F910895AF93BF93AFEE49
:100E2000B1E0EEE8F1E04D91EDDF4D91EBDF4D915A
:100E3000E9DFBF91AF91EEE8F1E078E121D00895CC
:100E4000AF93BF93A2EFB1E0EEE8F1E04D91DADFAE
:100E50004D91D8DF4D91D6DFBF91AF91EEE8F1E033
:100E600078E10ED00895E6EFF1E07081772319F470
:100E7000EFEAF1E002C0EFECF1E070E201D008959A
:100E80003F934F937F9331913323E1F400008A9A8B
:100E900044E14A95F1F700008A9844E04A95F1F759
:100EA0007A9589F7000000000000000000000000B3
:100EB0008A9A48E04A95F1F700008A987F914F910D
:100EC0003F9108958A9A46E04A95F1F700000000A4
:100ED0008A9842E14A95F1F7000000007A9599F668
:100EE0000000000000000000000000008A9A44E0BA
:100EF0004A95F1F700008A987F914F913F910895AC
:100F0000FC0120812F3F59F0332727FD309526170C
:100F1000370719F4FC01418308950296F1CF089533
:100F2000FC012081223011F48181089580E0089530
:100F3000FC018081833031F0843059F0813069F4D4
:100F4000818108958281918187FD05C098172CF0D9
:100F500006C091818281891714F480E0089581E0B0
:100F60000895CF92DF92EF92FF920F931F93CF934A
:100F7000DF938C017B016A019A012C5F3F4FF901DD
:100F800034978081882311F1F9013197808132975C
:100F90008083F3CFF8019181E601F4E09F02C00D58
:100FA000D11D112498819230B1F09330F9F0913035
:100FB00059F4970144E08402200D311D1124C90128
:100FC000B7DF9981982B99830E5F1F4FF8018081BD
:100FD0008F3F01F718C0F70194E08902E00DF11D81
:100FE00011248081823081F781810BC0F70124E0D8
:100FF0008202E00DF11D1124CF019ADF882321F335
:101000008A818983E1CFDF91CF911F910F91FF906A
:10101000EF90DF90CF90089581E88FBD8AE08EBD7C
:101020001BBC8FE18ABD0895C198B99A0895CF93EA
:10103000DF93EC01F1DF2FEF8BED95E02150804045
:101040009040E1F700C000001FBC2FEF80E792E066
:10105000215080409040E1F700C000002197209788
:1010600049F7DF91CF910895892B11F41FBC0895A2
:10107000D3CF1F920F920FB60F9211248F938091AE
:10108000F7018C3318F48F5F8093F7018F910F90E5
:101090000FBE0F901F90189589B78E7F89BF089556
:1010A00089B7816089BF089585E083BF12BE89B783
:1010B000816089BF1092F70108958091F7018C3308
:1010C00020F01092F70181E0089580E0089549E052
:1010D00051E060E070E08EE392E0DEC249E051E072
:1010E00060E070E08EE392E0C7D247E050E06EE649
:1010F00071E08EE392E0ACD20097B9F087E0EEE6C3
:10110000F1E0AEE3B2E001900D928A95E1F7109222
:1011100045021092460240E051E06FEF70E087E434
:1011200092E0A3D2D4DF81E090E008951FBC83E079
:101130008EBD1DBC1CBC1092F90186ED96E090930B
:10114000FB018093FA01089508B602FE0AC088B731
:10115000846088BF86ED96E09093FB018093FA014E
:1011600026C08CB59DB5893E23E0920758F1873D96
:1011700026E0920720F18E5E92409093FB018093CF
:10118000FA018091FA019091FB01883E934030F47E
:1011900086ED96E09093FB018093FA011092F8019E
:1011A0001DBC1CBC88B7846088BF1092F9011DBCAF
:1011B0001CBC88B7846088BF1092F901089586ED41
:1011C00096E0DBCF8091F8018F5F8093F801893042
:1011D00070F31DBC1CBC88B7846088BF81E090E0C0
:1011E0009093FB018093FA011092F801DECF809179
:1011F000F90181110DC02CB53DB58091FA01909196
:10120000FB012817390720F081E08093F901089548
:1012100080E00895A398AB98BC9AC49808950F9362
:101220001F93CF93DF93662309F454C07727A0E080
:10123000B0E040E050E09D0146175707ACF4189627
:1012400010E8FC01E40FF51F00810123E901C95BEF
:10125000DC4F08832F5F3F4F16952A173B07A1F7F6
:101260004F5F5F4FD901E7CFE7E4F3E0CF93DF9320
:10127000EF93FF930191002311F069F41BC000006C
:10128000A39A1DE014D0A398000000000000000005
:10129000119781F70FC0A39A12E0000008D0A3981D
:1012A00019E005D000000000119721F703C01A953E
:1012B000F1F7089500000000FF91EF91DF91CF91C9
:1012C000A39A12E00000F3DFA3980FEF0A9511F044
:1012D0009B9BFCCFE7E4F3E0EF93FF9344270027C9
:1012E0000395A1F09B99FCCF08C00BE4039572F025
:1012F0009B99FCCF439551F001930BE4039532F099
:101300009B9BFCCF439511F00193EFCFFF91EF91A1
:10131000842F90E00097C1F040FF16C0DF019D01CF
:101320007081618151E0761708F050E05D9332964C
:101330005A2F521B5417A0F32AE12A95F1F700C047
:1013400001979595879502C080E090E0DF91CF915D
:101350001F910F910895CF93DF931F92CDB7DEB702
:10136000198261E070E0CE01019659DF0097F1F03B
:101370004897F9F480914B03811188E090914C03D8
:101380009111846090914D039111826090914E0370
:10139000911181608A3038F4883070F4853049F4D6
:1013A00081E090E00BC08B3039F003C080E090E02A
:1013B00005C083E090E002C082E090E00F90DF91F2
:1013C000CF910895CF93DF931F92CDB7DEB7BDDCE9
:1013D0009093FD018093FC0111BA82B38B6F82BBA5
:1013E000889A14BA8FEF85BB85B7886085BF85B7AB
:1013F0008B7F85BF8BB780648BBF80E2EFEAF1E023
:10140000DF01282F1D922A95E9F7EFECF1E0DF01CB
:101410001D928A95E9F785E08093EF011092F00123
:1014200092E09093F1018093F2011092F3011092F7
:10143000F401FADD81E090E0FADD50DE892B19F04D
:1014400082E090E0F4DD78948091450290E066D8E7
:101450002BDEE091FC01F091FD010284F385E02D8B
:101460000995909ABFEFE9E6F8E1B150E040F0400D
:10147000E1F700C00000E091FC01F091FD0104845F
:10148000F585E02D81E00995882329F08FEF99EF0C
:101490000197F1F7EECFE091FC01F091FD0100889A
:1014A000F189E02D8EEF91E00995AFEFB9EF11973B
:1014B000F1F700C000008091FE01805880937D010B
:1014C0008091FF01805880937C01A7D68091BB005A
:1014D000882319F08EEA90E030D9909827DE10E04A
:1014E0008091F501882319F01092F5012DDE7FDE41
:1014F0008823B1F3909AD0DDE091FC01F091FD01D9
:101500000484F585E02D80E009958983C9DD9098F4
:101510008981882339F01F5F15312CF081E090E03C
:1015200086DDA9CF10E0E091FC01F091FD01068479
:10153000F785E02D0995882339F1909AE091FC0117
:10154000F091FD010088F189E02D8EEF91E0099581
:1015500064D64AE151E06EEA70E086E092E001DD97
:101560008091F601882319F06FEA71E002C06FECF8
:1015700071E08AE191E0C6D99091F60181E0911184
:1015800080E08093F60190988EEA90E090D9A8CF01
:10159000052E97FB16F400940FD057FD05D020D0F0
:1015A00007FC02D046F408C050954095309521952F
:1015B0003F4F4F4F5F4F089590958095709561957F
:1015C0007F4F8F4F9F4F08952DD0B7FF0895821BF7
:1015D000930B0895B7FF32C031D0821B930B08954F
:1015E000A1E21A2EAA1BBB1BFD010DC0AA1FBB1F27
:1015F000EE1FFF1FA217B307E407F50720F0A21B99
:10160000B30BE40BF50B661F771F881F991F1A9405
:1016100069F760957095809590959B01AC01BD012F
:10162000CF010895A29FB001B39FC001A39F01D035
:10163000B29F700D811D1124911D0895F3DFA59FA8
:10164000900DB49F900DA49F800D911D11240895BD
:10165000FB01DC0104C08D910190801921F44150FF
:101660005040C8F7881B990B0895DC0101C06D93A9
:1016700041505040E0F70895DC01CB01FC01E199B5
:10168000FECF06C0FFBBEEBBE09A31960DB20D92C5
:1016900041505040B8F70895DC01CB0102C02D91B4
:1016A00005D041505040D8F70895262FE199FECF3C
:1016B0009FBB8EBB2DBB0FB6F894E29AE19A0FBE8A
:0816C00001960895F894FFCF94
:1016C80000000101020203030404050506060707DA
:1016D800080809090A0A0B0B0C0C0D0D0E0E0F0F4A
:1016E80010141114121413141414151416141714B6
:1016F800181419141A14FFFF010008000000000054
:10170800000000009C0664063605220595060100C7
:1017180000000100000001000000010000000100BD
:101728000000010000000300E000030020000300A7
:10173800E00003002000010000000100000001009B
:10174800000001000000020000000200000001008B
:101758000000010000000300E00003002000030077
:10176800E000030020000400200004002000020024
:10177800000002000000000000000100000001005D
:10178800000001000000010000000100000001004D
:10179800000001000000010000000100000001003D
:1017A800000001000000010000000100000001002D
:1017B8000000020000000200000003008100030096
:1017C8007F000300810003007F0000000000474302
:0817D800324E36347636000073
:00000001FF
